:100000000C9477000C94780D0C94A50D0C949F0023
:100010000C949F000C949F000C949F000C949F00E4
:100020000C949F000C949F000C949F000C949F00D4
:100030000C949F000C949F000C949F000C949F00C4
:100040000C94D20D0C94B3000C9411100C94581015
:100050000C949F000C949F000C949F000C949F00A4
:100060000C94A60B0C949F00486F6C6964617944F2
:1000700075696E6F30372D323000486F6C6964617E
:10008000794475696E6F30372D3230000000000002
:10009000240027002A0000000000250028002B0073
:1000A00000000000230026002900040404040404C6
:1000B0000404020202020202030303030303010217
:1000C00004081020408001020408102001020408E6
:1000D00010200000000700020100000304060000D9
:1000E000000000000000110196091D0A8C11112466
:1000F0001FBECFEFD8E0DEBFCDBF11E0A0E0B1E082
:10010000E2EFFAE202C005900D92AA34B107D9F7E6
:1001100016E0AAE4B1E001C01D92A133B107E1F7F6
:1001200010E0CEEED0E004C02297FE010E947315CD
:10013000C63ED107C9F70E94E2110C9477150C94C2
:100140000000DC0101C06D9341505040E0F708957C
:10015000FC01A081B1812D913C91F901099508958F
:1001600081E0089508951F920F920FB60F92112407
:100170002F933F934F935F936F938F939F93EF933F
:10018000FF936EB58091710490E04091030150910E
:1001900004019A01220F331F240F351F8217930782
:1001A00074F480917104E0913804F0913904E80FFF
:1001B000F11D6083809171048F5F80937104FF91C2
:1001C000EF919F918F916F915F914F913F912F91FF
:1001D0000F900FBE0F901F901895FC01549A80E16C
:1001E00082838BE290E0948383830895DF93CF939F
:1001F00000D00F92CDB7DEB7DC01AB01ED91FC91E1
:100200000680F781E02D19821A821B82BE016F5F82
:100210007F4F20E009950F900F900F90CF91DF91C5
:10022000089508950E94170E6093090170930A01C2
:1002300080930B0190930C0108951F93809103010B
:1002400090910401892B09F443C082E00E94BD0F04
:10025000892B49F4809172048823D1F5109271049E
:1002600088E060E033C08091710490E04091030128
:10027000509104019A01220F331F240F351F82175A
:10028000930724F480913C048823E1F011E010935B
:100290003A040E94170E20916304309164044427AD
:1002A00037FD4095542F260F371F481F591F2093A5
:1002B0006D0430936E0440936F0450937004109358
:1002C000720406C01092710488E061E00E94690F18
:1002D0001F9108958EE480937C0062E070E080E0DE
:1002E00090E00E94980E80917A00806480937A005A
:1002F00080917A0086FDFCCF8091780090E0A0E0AC
:10030000B0E060917900362F20E0442737FD40951A
:10031000542F282B392B4A2B5B2B60E070E381E1B3
:1003200090E00E944215CA01B90108950F931F93EE
:100330008C0184E095E060E570E00E94B209612FD5
:10034000772767FD7A9584E095E00E94650A107032
:1003500084E095E0602F0E94650A84E095E00E94A9
:10036000A80A84E095E060E570E041E050E00E947A
:10037000B90A84E095E00E94BC09892B11F480E061
:1003800004C084E095E00E94C5091F910F91089573
:10039000DF92EF92FF920F931F938C01D62E84E091
:1003A000E82E85E0F82EC70160E570E00E94B209F2
:1003B000612F772767FD7A95C7010E94650A107043
:1003C000C701602F0E94650AC7016D2D0E94650A52
:1003D000C7010E94A80A65E070E080E090E00E94FA
:1003E000980E1F910F91FF90EF90DF9008950F935B
:1003F0001F93CF93DF93182F8F3339F48BE895E059
:1004000068E670E00E94691293C18B3519F08D3552
:1004100081F407C084E095E068E070E00E94DC0AA7
:1004200004C084E095E00E94BD0A8BE895E0612F4E
:100430007DC1813491F4809167048370825F60E0B4
:100440000E942A0F8091670483700E94080F809198
:10045000670483700E94080FC2C0823479F585E07A
:100460000E94BD0F8C0186E00E94BD0F892B19F000
:10047000C0E0D0E002C0C2E0D0E087E00E94BD0F43
:10048000892B19F020E030E002C024E030E060E089
:1004900070E0012B11F461E070E080913E04992737
:1004A00087FD909544E0880F991F4A95E1F7682BE6
:1004B000792B6C2B7D2B622B732B2CC18334F9F49D
:1004C0008091650490916604029771F46091050132
:1004D0007091060180916704909168040E940D1547
:1004E000609169040E94C801609105017091060144
:1004F00080916704909168040E940D151FC0843498
:1005000039F580913D0490E02091650430916604B6
:1005100082239323892B81F0609167047091680492
:100520008091410490914204681779070CF060E0D3
:1005300085E090E00E94C80185E090E00E9496016D
:10054000682F8BE895E04AE050E00E942413F0C049
:100550008534B1F48091650490916604892B59F03B
:1005600010923B048091670490916804892B19F0E4
:1005700081E080933B0460E070E080913B04A4C084
:10058000873469F4809167048370825F61E00E9420
:100590002A0F809167048370825F60E00EC0883408
:1005A00079F4809167048370825F61E00E942A0F72
:1005B000809167048370825F61E00E94690F09C0C7
:1005C000893479F4809167048370825F60E00E94CF
:1005D0002A0F809167048370825F0E94BD0FBC0167
:1005E00099C08C3401F58091650490916604892B43
:1005F000A9F080913D04882389F06091670470918F
:1006000068046B3F710514F06AEF70E070930401A9
:100610006093030183E090E00E94C80160910301B0
:100620007091040177C0803599F4809165049091B0
:100630006604892B41F0809167049091680490933F
:10064000400480933F0460913F047091400462C075
:10065000823519F58091650490916604029781F4C2
:10066000E0916704F0916804EF70F070EE0FFF1FE7
:10067000ED5BFB4F8091690490916A0491838083C4
:10068000E0916704F0916804EF70F070EE0FFF1FC7
:10069000ED5BFB4F608171813DC08435D1F4809169
:1006A000650490916604892B59F010923C04809166
:1006B000670490916804892B19F081E080933C04D1
:1006C00060E070E080913C04882321F161E070E0FB
:1006D00021C0863559F40E946A01AB01BC018BE848
:1006E00095E02AE030E00E94821322C08735C9F4E9
:1006F0008091650490916604892B41F08091670494
:1007000090916804909364048093630460916304FF
:10071000709164048BE895E04AE050E00E949613E3
:1007200007C080322CF08BE895E06FE30E947D12C9
:10073000DF91CF911F910F9108950F931F93CF9346
:10074000DF938BE895E040E052EC61E070E00E94BE
:10075000881085E062E00E942A0F86E062E00E9435
:100760002A0F87E062E00E942A0F88E061E00E9481
:100770002A0F88E061E00E94690F8CE061E00E942E
:100780002A0F8CB580648CBDC0910301D091040107
:100790001C161D06D4F4009128011091290189E04E
:1007A00090E00E94F111FC011582168217821086DA
:1007B00088E191E091838083C801BF014AE451E060
:1007C0009E0100E010E00E94F3088AE491E090931B
:1007D000390480933804109271041092720480E0FE
:1007E0006DE171E041E050E00E94550D81E062E171
:1007F00071E042E050E00E94550D8CB580688CBDE0
:1008000085E00E94BD0F892B29F480913E048F5F03
:1008100080933E0486E00E94BD0F892B29F48091CD
:100820003E048E5F80933E0487E00E94BD0F892BBB
:1008300029F480913E048C5F80933E0484E095E02F
:100840000E94BD0A80E090E00E949601883669F51A
:1008500081E090E00E949601813039F580933D045B
:1008600082E090E00E94960190E0880F991F880F27
:10087000991F909306018093050183E090E00E9408
:100880009601809303011092040184E090E00E949D
:100890009601809341041092420485E090E00E940A
:1008A000960180933F04109240048BE895E06AE73C
:1008B00070E00E946912DF91CF911F910F9108950E
:1008C0000F931F938C010E94250E9B01AC01F80130
:1008D00080819181A281B381281B390B4A0B5B0B6C
:1008E000223331054105510534F482E390E0821B47
:1008F000930B0E944D0E1F910F910895CF92DF929E
:10090000EF92FF920F931F93CF93DF936C01162FFB
:10091000072FEA01E22E05960E946004F894212F29
:10092000302FC901FC01BE01660F771F6C0F7D1FC0
:10093000680F791F5BB150618BB18F7E8BB92181BC
:100940003E2D239F212DCCC095E05BB902E00A9596
:10095000F1F727FF8BB90014001402E00A95F1F7B4
:100960008BB9001400140014220F915071F7001479
:100970005BB902E00A95F1F727FF8BB90014001468
:1009800002E00A95F1F78BB902E00A95F1F700143D
:100990005BB902E00A95F1F726FF8BB90014001449
:1009A00002E00A95F1F78BB9001430814E2D349F87
:1009B000312D5BB902E00A95F1F725FF8BB90014E0
:1009C000001402E00A95F1F78BB902E00A95F1F7FD
:1009D00095E05BB902E00A95F1F737FF8BB9001497
:1009E000001402E00A95F1F78BB90014001400140A
:1009F000330F915071F700145BB902E00A95F1F7DB
:100A000037FF8BB90014001402E00A95F1F78BB997
:100A100002E00A95F1F700145BB902E00A95F1F7DC
:100A200036FF8BB90014001402E00A95F1F78BB978
:100A3000001442812E2D429F412D5BB902E00A95A0
:100A4000F1F735FF8BB90014001402E00A95F1F7B5
:100A50008BB902E00A95F1F795E05BB902E00A95DF
:100A6000F1F747FF8BB90014001402E00A95F1F783
:100A70008BB9001400140014440F915071F7001446
:100A80005BB902E00A95F1F747FF8BB90014001437
:100A900002E00A95F1F78BB9001400140014001459
:100AA000001433965BB902E00A95F1F746FF8BB963
:100AB0000014001402E00A95F1F78BB900142181AB
:100AC0003E2D239F212D5BB902E00A95F1F745FFEA
:100AD0008BB90014001402E00A95F1F78BB90014E9
:100AE000E617F70708F430CF1124E0908605F09060
:100AF00087050091880510918905BE01F5E0660F14
:100B0000771FFA95E1F7CC0FDD1F6C1B7D0B882753
:100B100077FD8095982F28EE33E040E050E00E946A
:100B20004215E20EF31E041F151FE0928605F09297
:100B30008705009388051093890578940E94250EF7
:100B4000F6016583768387839087DF91CF911F912C
:100B50000F91FF90EF90DF90CF900895BF92CF92CA
:100B6000DF92EF92FF920F931F93CF93DF936C016D
:100B70007B01EA01122F05960E946004F894BE01E1
:100B8000660F771F6C0F7D1F6E0D7F1D5BB150616F
:100B90008BB18F7E8BB9D7011196BC902B2D219FE5
:100BA000212DF701CFC095E05BB902E00A95F1F77E
:100BB00027FF8BB90014001402E00A95F1F78BB9F6
:100BC000001400140014220F915071F700145BB947
:100BD00002E00A95F1F727FF8BB90014001402E038
:100BE0000A95F1F78BB902E00A95F1F700145BB9A9
:100BF00002E00A95F1F726FF8BB90014001402E019
:100C00000A95F1F78BB90014D7013C910014319F7C
:100C1000312D5BB902E00A95F1F725FF8BB900147D
:100C2000001402E00A95F1F78BB902E00A95F1F79A
:100C300095E05BB902E00A95F1F737FF8BB9001434
:100C4000001402E00A95F1F78BB9001400140014A7
:100C5000330F915071F700145BB902E00A95F1F778
:100C600037FF8BB90014001402E00A95F1F78BB935
:100C700002E00A95F1F700145BB902E00A95F1F77A
:100C800036FF8BB90014001402E00A95F1F78BB916
:100C90000014D70112964C910014419F412D5BB96D
:100CA00002E00A95F1F735FF8BB90014001402E059
:100CB0000A95F1F78BB902E00A95F1F795E05BB977
:100CC00002E00A95F1F747FF8BB90014001402E027
:100CD0000A95F1F78BB9001400140014440F9150D9
:100CE00071F700145BB902E00A95F1F747FF8BB981
:100CF0000014001402E00A95F1F78BB900140014F7
:100D000000140014001433965BB902E00A95F1F761
:100D100046FF8BB90014001402E00A95F1F78BB975
:100D2000001400142B2D219F212D5BB902E00A95A0
:100D3000F1F745FF8BB90014001402E00A95F1F7B2
:100D40008BB90014E617F70708F42DCF1124E090B3
:100D50008605F09087050091880510918905BE01F0
:100D600085E0660F771F8A95E1F7CC0FDD1F6C1BBE
:100D70007D0B882777FD8095982F28EE33E040E0A3
:100D800050E00E944215E20EF31E041F151FE09270
:100D90008605F0928705009388051093890578945D
:100DA0000E94250EF6016583768387839087DF9105
:100DB000CF911F910F91FF90EF90DF90CF90BF9058
:100DC00008951F93182F682F62956F7060636A33C0
:100DD0000CF0695D772767FD70958BE895E00E94C0
:100DE0005011612F6F7060636A330CF0695D772773
:100DF00067FD70958BE895E00E9450111F91089552
:100E0000EF92FF920F931F93CF93DF938BE895E0C0
:100E10000E940611892B09F483C081E080933A0473
:100E20000E94170E2091630430916404442737FD1B
:100E30004095542F260F371F481F591F20936D04CC
:100E400030936E0440936F04509370048BE895E0E8
:100E50000E942211182F80913B04882329F08BE8EF
:100E600095E0612F0E944112812F80538A3058F5FE
:100E70008091650490916604892B31F481E090E0C3
:100E80009093660480936504E0916504F091660494
:100E9000EE0FFF1FEB59FB4F808191819C0153E0C6
:100EA000220F331F5A95E1F7880F991F280F391F1A
:100EB00020533040812F992787FD9095280F391FA7
:100EC000318320832DC01C3201F5809165049091FF
:100ED000660482309105CCF4892B31F481E090E0F6
:100EE0009093660480936504E0916504F091660434
:100EF0003196F0936604E09365043197EE0FFF1F7F
:100F0000E959FB4F118210820BC0812F0E94F7011B
:100F1000109266041092650410926804109267049F
:100F200080913A04882309F0DDC0E0906D04F090D0
:100F30006E0400916F04109170040E94170E6E15DC
:100F40007F058007910708F4CDC08091030190913F
:100F50000401FC01EE0FFF1FE80FF91F2AE431E046
:100F6000C90160E070E0AF010E94A100E0900901BA
:100F7000F0900A0100910B0110910C0188EE93E0B2
:100F8000A0E0B0E0E80EF91E0A1F1B1F0E94170E1A
:100F9000E616F7060807190720F48FE380934A0145
:100FA00003C08FE380934C0185E00E94BD0F892B25
:100FB00029F480914C01815C80934C0186E00E9471
:100FC000BD0F892B29F480914C01815C80934C01E9
:100FD00087E00E94BD0F892B29F480914C01815C30
:100FE00080934C0120916B0430916C04237030701D
:100FF0002130310599F022303105F1F0809107015F
:1010000090910801232B29F5FC01EE0FFF1FE80F3B
:10101000F91FE65BFE4F8FEF808326C080910701AA
:1010200090910801FC01EE0FFF1FE80FF91FE65B2E
:10103000FE4F8FEF818318C08091070190910801C6
:10104000FC01EE0FFF1FE80FF91FE65BFE4F8FEF6D
:101050000AC0FC01EE0FFF1FE80FF91FE65BFE4F11
:101060008FEF8083818382838091030190910401BB
:101070001816190654F4E0912601F0912701CF01CA
:10108000EE5BFF4F60810E944809809107019091BB
:1010900008010196909308018093070120910301B4
:1010A00030910401821793077CF081E090E09093E7
:1010B00008018093070180916B0490916C04019664
:1010C00090936C0480936B040E94170E6E5C7F4FAC
:1010D0008F4F9F4F60936D0470936E0480936F04E5
:1010E0009093700480917204882309F459C0809110
:1010F0003C048823F1F1C0E0D0E011C0209729F032
:101100008BE895E06CE20E944112E0913804F09186
:101110003904EC0FFD1F80810E94E1062196809129
:10112000710490E0C817D9074CF38BE895E060E0B4
:1011300071E00E94B5130EC080917104E0913804F3
:10114000F0913904E80FF11D1082809171048F5FD6
:10115000809371048091710490E04091030150915B
:1011600004019A01220F331F240F351F82179307A2
:101170001CF380910301909104011816190654F490
:10118000E0912601F0912701CF01EE5BFF4F6081D6
:101190000E9448091092720488E061E00E94690F81
:1011A000809163049091640418161906ACF4809140
:1011B0003A04882389F0E0906D04F0906E04009169
:1011C0006F04109170040E94170E6E157F05800742
:1011D000910710F010923A04DF91CF911F910F9177
:1011E000FF90EF900895DF92EF92FF920F931F937D
:1011F000CF93DF93EC017B01101611062CF0D22E59
:10120000032F20E030E002C0D02E012FC05CDF4F62
:10121000A881B981C054D040FE0160E070E007C0F1
:10122000808191813896892B41F06F5F7F4F6A17DB
:101230007B07B4F3EE24FF2422C0E3E0660F771FA0
:10124000EA95E1F7DE01A60FB71F1196FC92EE9228
:10125000FE01E60FF71F5383428317963C932E93AC
:101260001697FB013496EC0FFD1FD0820183D70146
:10127000ED91FC910190F081E02DC7010995C70126
:10128000DF91CF911F910F91FF90EF90DF90089524
:10129000DF92EF92FF920F931F93CF93DF93D62E9F
:1012A000EC0100E010E050E4E52EF12CE80EF91E10
:1012B0001DC0A881B9811097F9F0ED91FC911197AB
:1012C0002E813F81C901880F991F820F931F6A8168
:1012D0007B81680F791F4C815D810084F185E02D51
:1012E000CD012D2D09950F5F1F4F2896F7018081A5
:1012F000918108171907ECF2DF91CF911F910F919F
:10130000FF90EF90DF900895FC01E05CFF4F88E0D4
:1013100090E0819391938FEF8083E254F040CF016E
:1013200060E040E450E00E94A709089583E794E05C
:101330000E94840980EE92E3ACE1B0E08093B604B1
:101340009093B704A093B804B093B9040895DC0156
:1013500040FF03C001C06D936D934250E0F75040D1
:10136000D0F7089581E08093FF046093DC0410922D
:10137000FD041092FE0408952091DB0430E080917A
:10138000DA04281B3109C90108954091DA048091DB
:10139000DB04481718F02FEF3FEF0AC0E42FF0E00E
:1013A000E654FB4F8081282F30E04F5F4093DA04F2
:1013B000C9010895E091DA048091DB04E81718F080
:1013C000EFEFFFEF06C0F0E0E654FB4F8081E82F1F
:1013D000F0E0CF0108950895AC012091020530910D
:1013E000030521153105E1F09091DA048091DB04C9
:1013F0009817B0F090E008C0FA01EA0FFB1F808157
:10140000A654BB4F8C939F5FA92FB0E0A617B707D8
:101410009CF31092DA046093DB04CB01F901099587
:101420000895E0910005F0910105309729F01092A0
:10143000FD041092FE04099508951092070510927C
:10144000060588EE93E0A0E0B0E080930805909355
:101450000905A0930A05B0930B058EE291E09093E5
:101460000505809304050895CF92DF92EF92FF92D5
:101470000F931F93CF93DF937C016B018A018091BF
:10148000FF048823A1F0C0E0D0E00DC0D701ED91AA
:10149000FC91D601AC0FBD1F0190F081E02DC7017A
:1014A0006C9109952196C017D10780F304C0CB0138
:1014B000642F0E94810BC801DF91CF911F910F9182
:1014C000FF90EF90DF90CF900895DF93CF930F922E
:1014D000CDB7DEB7FC0169838091FF048823C9F092
:1014E0008091FE04803238F081E090E09383828323
:1014F00020E030E015C08091FD04E82FF0E0E352D9
:10150000FB4F998190838F5F8093FD048093FE044D
:1015100005C0CE01019661E00E94810B21E030E020
:10152000C9010F90CF91DF9108950F93062F8091FD
:10153000DC046DED74E04091FE0421E00E942C0B70
:101540001092FD041092FE041092FF040F91089572
:1015500061E00E94950A0895413208F040E2862F2A
:101560006AEB74E00E94E30A1092DA048093DB04D1
:10157000089521E00E94AC0A08951092DA041092B6
:10158000DB041092FD041092FE040E94370D0895B2
:101590000F931F938C01862F0E94DF0A81E19AE04E
:1015A0000E94A10B8CEE99E00E949C0BC8010E9446
:1015B000BD0A1F910F9108950E94C80A0895880FCF
:1015C0008093BA000895382F413210F040E042C0B5
:1015D000809110058823E1F791E090931005209306
:1015E00012058FEF80937D0510923805415040938E
:1015F00039054F5F9093110580911105330F832BAF
:101600008093110580911305813041F410921305E8
:10161000809111058093BB0085EC01C085EE80931D
:10162000BC00809110058130E1F38091380584176A
:1016300010F44091380520E030E00AC0FB01E20FD1
:10164000F31FD901A85EBA4F8C9180832F5F3F4F63
:101650002417A0F3842F08950F931F93582F122F50
:10166000413210F081E04AC0809110058823E1F7F3
:1016700082E080931005009312058FEF80937D0523
:101680001092380540933905A8E1B5E0FB0102C08E
:1016900081918D938E2F861B8417D0F310921105A4
:1016A00080911105550F852B8093110580911305AD
:1016B000813041F410921305809111058093BB0095
:1016C00085EC01C085EE8093BC00112321F0809150
:1016D00010058230E1F380917D058F3F11F480E0A9
:1016E0000DC080917D05803211F482E007C08091A9
:1016F0007D05803311F084E001C083E01F910F91DC
:101700000895482F613210F081E00895809110050E
:10171000843011F082E0089560935B05AAE3B5E0A0
:10172000842F9C01F90102C081918D938E2F841B1F
:101730008617D0F380E008959093170580931605DF
:101740000895909315058093140508951F920F92A4
:101750000FB60F9211242F933F934F935F936F9384
:101760007F938F939F93AF93BF93EF93FF9380915A
:10177000B90090E0887F90708036910509F4F2C03E
:1017800081369105CCF58832910509F47BC0893208
:101790009105B4F48031910509F46FC08131910550
:1017A0003CF4009709F447C1089709F04FC165C0A0
:1017B0008831910509F466C0809709F047C182C05D
:1017C0008034910509F4A4C08134910544F4803338
:1017D000910509F482C0C89709F038C189C08035E5
:1017E000910509F489C08835910509F496C08834BB
:1017F000910509F02BC1AEC08839910509F413C1D8
:1018000089399105ECF48837910509F4ABC0893723
:1018100091054CF48836910509F4A4C080379105F0
:1018200009F014C19FC08838910509F4FCC08039C3
:10183000910509F49DC08038910509F007C198C051
:10184000803B910509F4C6C0813B91054CF4803A78
:10185000910509F49FC0883A910509F0F7C0BAC014
:10186000803C910509F4E3C0883C910509F4DFC090
:10187000883B910509F0EAC0C2C0809111058093B0
:10188000BB00CFC09091380580913905981768F456
:1018900090913805E92FF0E0E85EFA4F808180935F
:1018A000BB009F5F90933805BCC0809112058823D0
:1018B00009F44BC085ED8093BC008091BC0084FD91
:1018C000FCCFC2C080E280937D0585ED8093BC0093
:1018D0008091BC0084FDFCCFB7C080E380937D0580
:1018E00085ED8093BC008091BC0084FDFCCFACC032
:1018F00088E380937D059BC0809138059091BB0063
:10190000E82FF0E0E85EFA4F90838F5F8093380510
:10191000909138058091390582C080913805909169
:10192000BB00E82FF0E0E85EFA4F90838F5F809372
:10193000380580911205882341F085ED8093BC0025
:101940008091BC0084FDFCCF7FC081E080931305B3
:1019500084EA6EC085ED8093BC008091BC0084FD5C
:10196000FCCF72C083E08093100510927C0559C0B3
:1019700080917C05803208F056C080917C05909162
:10198000BB00E82FF0E0E45AFA4F90838F5F80931A
:101990007C0547C080917C05803230F4E0917C0565
:1019A000F0E0E45AFA4F108285ED8093BC008091FC
:1019B000BC0084FDFCCF1092100560917C05E09185
:1019C0001605F09117058CE595E070E009951092E9
:1019D0007C052DC084E08093100510925A0510926A
:1019E0005B05E0911405F0911505099580915B0563
:1019F000882329F481E080935B0510923A05909149
:101A00005A05E92FF0E0E65CFA4F80818093BB0035
:101A10009F5F90935A0590915A0580915B059817A6
:101A200010F485EC01C085E88093BC000FC085EC04
:101A30008093BC0009C010927D0585ED8093BC00A9
:101A40008091BC0084FDFCCF10921005FF91EF91B6
:101A5000BF91AF919F918F917F916F915F914F91C6
:101A60003F912F910F900FBE0F901F9018951092DD
:101A7000100581E0809312051092130582E161E068
:101A80000E94690F83E161E00E94690FE9EBF0E0D9
:101A900080818E7F808380818D7F80838CE58093A1
:101AA000B80085E48093BC000895823000F5E82FEB
:101AB000F0E0EE0FFF1FE258FA4F71836083882336
:101AC00019F08130A1F408C0809169008C7F842BCB
:101AD00080936900E89A089580916900440F551F2A
:101AE000440F551F837F842B80936900E99A0895E2
:101AF0001F920F920FB60F9211242F933F934F9383
:101B00005F936F937F938F939F93AF93BF93EF9365
:101B1000FF9380917E0590917F05892B29F0E091BC
:101B20007E05F0917F050995FF91EF91BF91AF91EF
:101B30009F918F917F916F915F914F913F912F91E5
:101B40000F900FBE0F901F9018951F920F920FB617
:101B50000F9211242F933F934F935F936F937F9333
:101B60008F939F93AF93BF93EF93FF9380918005E3
:101B700090918105892B29F0E0918005F0918105F4
:101B80000995FF91EF91BF91AF919F918F917F91B7
:101B90006F915F914F913F912F910F900FBE0F90DA
:101BA0001F9018951F920F920FB60F9211242F932A
:101BB0003F938F939F93AF93BF93809186059091AE
:101BC0008705A0918805B091890530918A05232F5A
:101BD0002A592D3720F02D570196A11DB11D2093B4
:101BE0008A058093860590938705A0938805B09316
:101BF00089058091820590918305A0918405B0911B
:101C000085050196A11DB11D8093820590938305E2
:101C1000A0938405B0938505BF91AF919F918F915B
:101C20003F912F910F900FBE0F901F9018958FB777
:101C3000F894209186053091870540918805509150
:101C400089058FBFB901CA0108953FB7F894809103
:101C5000820590918305A0918405B091850526B5F4
:101C6000A89B05C02F3F19F00196A11DB11D3FBFD4
:101C7000BA2FA92F982F8827820F911DA11DB11D62
:101C80009C01AD01220F331F441F551F280F391F20
:101C90004A1F5B1FB901CA010895000000009C01A2
:101CA0002150304049F0220F331F220F331F03977A
:101CB000820F931F0197F1F70895789484B582609D
:101CC00084BD84B5816084BD85B5826085BD85B5E0
:101CD000816085BDEEE6F0E0808181608083E1E88F
:101CE000F0E01082808182608083808181608083C7
:101CF000E0E8F0E0808181608083E1EBF0E08081CA
:101D000084608083E0EBF0E0808181608083EAE79B
:101D1000F0E0808184608083808182608083808124
:101D2000816080838081806880831092C1000895E3
:101D3000EF92FF920F931F93CF93DF937B018C0160
:101D40009FB7F894209182053091830540918405D6
:101D50005091850586B5A89B06C08F3F21F02F5F67
:101D60003F4F4F4F5F4F9FBF542F432F322F22279C
:101D7000280F311D411D511DDA01C901880F991F1E
:101D8000AA1FBB1F820F931FA41FB51FEC0134C0F5
:101D90000E94ED149FB7F89420918205309183053D
:101DA000409184055091850586B5A89B06C08F3F5C
:101DB00021F02F5F3F4F4F4F5F4F9FBF542F432F57
:101DC000322F2227280F311D411D511DDA01C90173
:101DD000880F991FAA1FBB1F820F931FA41FB51F37
:101DE0008C1B9D0B885E934098F20894E108F108E3
:101DF00001091109C851DC4FE114F1040105110575
:101E000039F6DF91CF911F910F91FF90EF900895D8
:101E1000982F8E3008F09E50977080910D0182951A
:101E2000880F880F807C892B80937C0080917A00BA
:101E3000806480937A0080917A0086FDFCCF2091A7
:101E4000780040917900942F80E030E0282B392BE6
:101E5000C9010895CF93DF93482F50E0CA018254FF
:101E60009F4FFC01349146555F4FFA0184918823BE
:101E700069F190E0880F991FFC01E457FF4FA5918D
:101E8000B491FC01EA56FF4FC591D491662351F4F9
:101E90002FB7F8948C91932F909589238C938881F8
:101EA00089230BC0623061F42FB7F8948C91932F83
:101EB000909589238C938881832B88832FBF06C0BC
:101EC0009FB7F8948C91832B8C939FBFDF91CF9118
:101ED0000895482F50E0CA018E529F4FFC01249173
:101EE000CA0182549F4FFC01949146555F4FFA01FD
:101EF0003491332309F440C0222351F1233071F08F
:101F0000243028F42130A1F0223011F514C02630FD
:101F1000B1F02730C1F02430D9F404C080918000A2
:101F20008F7703C0809180008F7D8093800010C0E8
:101F300084B58F7702C084B58F7D84BD09C0809140
:101F4000B0008F7703C08091B0008F7D8093B00088
:101F5000E32FF0E0EE0FFF1FEA56FF4FA591B4917B
:101F60002FB7F894662321F48C919095892302C0B1
:101F70008C91892B8C932FBF0895682F70E0CB0133
:101F80008E529F4FFC012491CB0182549F4FFC0144
:101F9000449166557F4FFB019491992319F420E0F9
:101FA00030E03CC0222351F1233071F0243028F47A
:101FB0002130A1F0223011F514C02630B1F02730C5
:101FC000C1F02430D9F404C0809180008F7703C021
:101FD000809180008F7D8093800010C084B58F77C2
:101FE00002C084B58F7D84BD09C08091B0008F7719
:101FF00003C08091B0008F7D8093B000892F90E066
:10200000880F991F80569F4FFC01A591B4918C9128
:1020100020E030E0842311F021E030E0C901089590
:1020200008951F920F920FB60F9211242F933F9392
:102030004F938F939F93EF93FF938091C00082FD06
:1020400019C04091C6008091A905282F30E02F5F6C
:102050003F4F2F7330708091AA0590E02817390701
:1020600059F0E091A905F0E0E557FA4F42A320931B
:10207000A90502C08091C600FF91EF919F918F91B9
:102080004F913F912F910F900FBE0F901F90189579
:102090008091A9052091AA0590E0805C9F4F821B4A
:1020A00091098F739070892B11F00E941010089580
:1020B0001F920F920FB60F9211242F938F939F931D
:1020C000EF93FF939091AB058091AC05981731F495
:1020D0008091C1008F7D8093C10010C0E091AC055C
:1020E000F0E0E351FA4F20818091AC0590E0019639
:1020F0008F7390708093AC052093C600FF91EF9191
:102100009F918F912F910F900FBE0F901F90189558
:10211000AF92BF92DF92EF92FF920F931F93CF93F4
:10212000DF93EC017A018B01DD24D39491E0A92E99
:10213000B12CE889F989DD2069F0C5010C8C02C059
:10214000880F991F0A94E2F7808360E47BE48CE4B3
:1021500090E005C0108260EA75E286E290E0A80196
:1021600097010E9420152150304040405040569524
:1021700047953795279580E12030380720F0DD20FE
:1021800011F0DD24D6CFEC85FD853083EE85FF850B
:1021900020831D8EEA89FB89408121E030E0C9015E
:1021A000088C02C0880F991F0A94E2F7482B4083DD
:1021B000EA89FB894081C901098C02C0880F991FF7
:1021C0000A94E2F7482B4083EA89FB894081C901E0
:1021D0000A8C02C0880F991F0A94E2F7482B4083AB
:1021E000EA89FB8980810B8C02C0220F331F0A947D
:1021F000E2F7209528232083DF91CF911F910F9143
:10220000FF90EF90DF90BF90AF900895FC01268D76
:10221000878D30E0205C3F4F281B31092F733070D1
:10222000C9010895FC01968D878D981719F42FEF39
:102230003FEF06C0878DE80FF11D82A1282F30E007
:10224000C9010895DC015E969C915E975F968C9122
:102250005F97981719F42FEF3FEF10C05F968C919E
:102260005F97FD01E80FF11D92A15F968C915F973A
:102270008F5F8F735F968C93292F30E0C90108958B
:10228000DC015D968C915D97882339F05096ED9135
:10229000FC915197808186FFF9CF5D961C9208953D
:1022A000DC0190968C919097282F30E02F5F3F4F64
:1022B0002F73307091968C91919790E02817390781
:1022C000C9F390968C919097FD01E80FF11DEE599E
:1022D000FF4F608390962C9390975296ED91FC91CE
:1022E0005397208181E090E05B960C905B9702C051
:1022F000880F991F0A94E2F7282B208381E05D96CE
:102300008C935D975096ED91FC91519780818064FC
:10231000808381E090E0089510928E0510928D05E3
:1023200088EE93E0A0E0B0E080938F059093900555
:10233000A0939105B09392058EE391E090938C0564
:1023400080938B051092AC058091AC058093AB0512
:102350001092AA058091AA058093A90585EC90E0CA
:10236000909398058093970584EC90E090939A055C
:102370008093990580EC90E090939C0580939B0559
:1023800081EC90E090939E0580939D0582EC90E017
:102390009093A00580939F0586EC90E09093A20512
:1023A0008093A10584E08093A30583E08093A40536
:1023B00087E08093A50585E08093A60581E0809362
:1023C000A7050895CF93DF930E945D0E0E949D03A1
:1023D000C8E4D0E10E9400072097E1F30E94481072
:1023E000F9CF0E94B8130895CF92DF92EF92FF9237
:1023F0000F931F93CF93DF937C016B018A01C0E0A1
:10240000D0E00FC0D6016D916D01D701ED91FC9127
:102410000190F081E02DC7010995C80FD91F015027
:1024200010400115110571F7CE01DF91CF911F9179
:102430000F91FF90EF90DF90CF900895EF92FF9271
:102440000F931F93CF93DF937C018B01C0E0D0E00B
:10245000F8010F5F1F4F6491662359F0D701ED918A
:10246000FC910190F081E02DC7010995C80FD91F9B
:10247000EFCFCE01DF91CF911F910F91FF90EF90A1
:102480000895DC01ED91FC910190F081E02D09951A
:102490000895EF92FF920F931F938C01DC01ED9151
:1024A000FC910190F081E02D6DE009957C01D8014F
:1024B000ED91FC910190F081E02DC8016AE0099551
:1024C0009C012E0D3F1DC9011F910F91FF90EF90B0
:1024D0000895EF92FF920F931F937C010E941E12AA
:1024E0008C01C7010E9449129C01200F311FC901B4
:1024F0001F910F91FF90EF900895EF92FF920F932D
:102500001F937C01DC01ED91FC910190F081E02DA5
:1025100009958C01C7010E944912080F191FC801B3
:102520001F910F91FF90EF900895CF93DF93EC01EF
:102530006115710519F420E030E00FC0DB010D904A
:102540000020E9F71197A61BB70BE881F9810280FB
:10255000F381E02DAD0109959C01C901DF91CF9177
:1025600008954F925F927F928F929F92AF92BF9207
:10257000CF92DF92EF92FF920F931F93DF93CF934F
:10258000CDB7DEB7A1970FB6F894DEBF0FBECDBFB3
:102590002C01742ECB01223008F42AE019A231E27A
:1025A000C32ED12CCC0EDD1E822E9924AA24BB244E
:1025B000672D752FA50194010E94201579018A01CC
:1025C000C801B701A50194010E94EE14472D461BD6
:1025D0000894C108D1084A3014F4405D01C0495C38
:1025E000F6014083E114F1040105110521F07E2C70
:1025F0005F2DC801DDCFC201B6010E949512A196E0
:102600000FB6F894DEBF0FBECDBFCF91DF911F9103
:102610000F91FF90EF90DF90CF90BF90AF909F9081
:102620008F907F905F904F900895DC0121153105C8
:1026300041F4ED91FC910190F081E02D642F09951A
:1026400008950E94B1120895CF92DF92EF92FF9207
:102650000F931F936C01E62E9A01FF2400E010E017
:10266000B801A7010E9415138C01C6010E944912EE
:10267000080F191FC8011F910F91FF90EF90DF9075
:10268000CF900895CF92DF92EF92FF920F931F9316
:10269000CF93DF93EC016A017B012115310541F4F1
:1026A000E881F9810190F081E02D642F09951FC028
:1026B0002A303105D1F477FF17C0E881F981019004
:1026C000F081E02D6DE209958C0144275527BA0170
:1026D0004C195D096E097F09CE012AE00E94B112F2
:1026E0009801280F391F04C02AE00E94B1129C01F2
:1026F000C901DF91CF911F910F91FF90EF90DF9073
:10270000CF900895EF92FF920F931F937C010E9448
:1027100042138C01C7010E9449129C01200F311FF6
:10272000C9011F910F91FF90EF900895CF92DF9212
:10273000EF92FF920F931F936C017B019A01002788
:10274000F7FC0095102FB801A7010E9442138C01DD
:10275000C6010E944912080F191FC8011F910F914D
:10276000FF90EF90DF90CF9008950E94951208950A
:102770000F931F93CF93DF93BC018230910510F428
:1027800062E070E0E0912F06F091300640E050E00A
:10279000A0E0B0E024C08081918186179707D0F037
:1027A0008617970771F482819381109729F0139609
:1027B0009C938E9312972CC09093300680932F0693
:1027C00027C04115510519F08417950718F48D019C
:1027D000AC01EF01DF01828193819C01F901309707
:1027E000D1F641155105F9F0CA01861B970B8430CB
:1027F000910580F48A819B810115110521F0F80172
:102800009383828304C09093300680932F06FE0149
:10281000329645C0FE01E80FF91F6193719302974C
:10282000998388833CC080912D0690912E06892B38
:1028300041F4809110019091110190932E068093A4
:102840002D0640911201509113014115510541F49B
:102850004DB75EB780910E0190910F01481B590B47
:1028600020912D0630912E0624173507B0F4CA01A9
:10287000821B930B8617970780F0AB014E5F5F4F6B
:102880008417950750F0420F531F50932E06409324
:102890002D06F9016193719302C0E0E0F0E0CF01F1
:1028A000DF91CF911F910F910895CF93DF939C01FA
:1028B000009709F48FC0EC0122971B821A82609165
:1028C0002F06709130066115710581F48881998118
:1028D000820F931F20912D0630912E06281739075D
:1028E00039F5D0932E06C0932D0674C0DB0140E06D
:1028F00050E0AC17BD0708F1BB83AA83FE0121910C
:102900003191E20FF31FAE17BF0779F48D919C91BF
:102910001197280F391F2E5F3F4F39832883129656
:102920008D919C9113979B838A834115510571F476
:10293000D0933006C0932F064DC012968D919C9176
:102940001397AD01009711F0DC01D3CFDA01139694
:10295000DC93CE931297FA0121913191E20FF31F8C
:10296000CE17DF0769F488819981280F391F2E5F00
:102970003F4FFA01318320838A819B819383828335
:10298000E0E0F0E0DB0112968D919C9113970097A7
:1029900019F0BC01FD01F6CFAB014E5F5F4FDB01CB
:1029A0008D919C91840F951F20912D0630912E06BC
:1029B0002817390779F4309729F4109230061092CD
:1029C0002F0602C0138212824250504050932E06AE
:1029D00040932D06DF91CF9108950895629FD00115
:1029E000739FF001829FE00DF11D649FE00DF11DCA
:1029F000929FF00D839FF00D749FF00D659FF00D79
:102A00009927729FB00DE11DF91F639FB00DE11D65
:102A1000F91FBD01CF011124089597FB092E072648
:102A20000AD077FD04D049D006D000201AF4709562
:102A300061957F4F0895F6F7909581959F4F089582
:102A4000A1E21A2EAA1BBB1BFD010DC0AA1FBB1FB2
:102A5000EE1FFF1FA217B307E407F50720F0A21B24
:102A6000B30BE40BF50B661F771F881F991F1A9491
:102A700069F760957095809590959B01AC01BD01BB
:102A8000CF01089597FB092E05260ED057FD04D0DF
:102A9000D7DF0AD0001C38F4509540953095219529
:102AA0003F4F4F4F5F4F0895F6F790958095709583
:102AB00061957F4F8F4F9F4F0895AA1BBB1B51E11C
:102AC00007C0AA1FBB1FA617B70710F0A61BB70B9E
:102AD000881F991F5A95A9F780959095BC01CD0143
:102AE0000895EE0FFF1F0590F491E02D0994F894DE
:022AF000FFCF16
:102AF2000D0A0032002000010018FCFFFF018000D7
:102B02003106000000000000ED00A800F600AE054E
:102B12007E04B000B2007304730400000000650A72
:102B2200340ABC09C509DA09EB090000000050119A
:0A2B3200F4110611221112114011D6
:00000001FF
